TagPDF.com

pdf to tiff converter c#


convert pdf to tiff asp.net c#

pdf to tiff converter c#













pdf converter online software word, pdf js library port support, pdf best ocr pro text, pdf itextsharp read using vb.net, pdf .pdf application file web,



how to convert pdf to jpg in c# windows application, convert pdf to jpg c# itextsharp, convert pdf to jpg c# itextsharp, pdf to excel c#, how to download pdf file from gridview in asp.net using c#, how to convert pdf to jpg in c# windows application, convert pdf to image in asp.net c#, adobe pdf library c#, open pdf and draw c#, how to use pdfdocument class in c#, pdf free library c#, convert pdf to tiff image in c#, c# code to convert pdf to excel, itextsharp add annotation to existing pdf c#, c# convert pdf to tiff free library



microsoft azure pdf, how to download pdf file from gridview in asp.net using c#, mvc print pdf, how to generate pdf in mvc 4, asp.net pdf viewer annotation, asp.net c# pdf viewer control, generate pdf using itextsharp in mvc, pdf viewer in mvc c#, asp.net mvc 4 generate pdf, print mvc view to pdf



print code 39 barcodes excel, code 128 excel add in free, asp.net 2d barcode generator, qr code scanner java download,

c# convert pdf to tiff pdfsharp

Convert a PDF into a series of images using C# and GhostScript ...
4 Sep 2011 ... Article which describes how to use C# and GhostScript to convert PDF files into raster images for displaying in an application without requiring ...

c# convert pdf to tiff free

Convert PDF to TIFF image in C# and Visual Basic .NET with PDF ...
The scripts below demonstrate how to render PDF to TIFF image in C# and Visual Basic .NET using Bytescout PDF Renderer SDK. C#  ...


c# convert pdf to tiff pdfsharp,
pdf to tiff conversion c#,
convert pdf to multipage tiff c#,
convert pdf to tiff c# aspose,
c# convert pdf to tiff ghostscript,
convert pdf to tiff image in c#,
convert pdf to tiff c# pdfsharp,
convert pdf to tiff c#,
c# pdf to tiff pdfsharp,

The preceding sections have shown you many of the features available for querying inmemory data by using the extension methods for the Enumerable class de ned in the System.Linq namespace. The syntax makes use of several advanced C# language features, and the resultant code can sometimes be quite hard to understand and maintain. To relieve you of some of this burden, the designers of C# added query operators to the language to enable you to employ LINQ features by using a syntax more akin to SQL. As you saw in the examples shown earlier in this chapter, you can retrieve the rst name for each customer like this:

convert pdf to tiff c# aspose

How to Convert PDF File to TIFF Image File | C#.NET Programming ...
This C# sample takes a local PDF as an input file and shows how to use well-​developed .NET APIs to convert PDF file to TIFF images in C#.NET using PDF to​ ...

convert pdf to tiff c#

Convert PDF to multipage TIFF in C# .NET - Tallcomponents
Page.Draw. Another way to convert PDF to TIFF using C# , is to use Page.Draw() to create a bitmap for each page, and then use standard .Net methods to write these to a tiff file. There are two issue with this though: .NET does not support creating a graphics instance for a monochrome bitmap.

5

public partial class Error404 : System.Web.UI.Page { protected void Page_Load(object sender, EventArgs e) { var errPath = "<i>No error path information is available.</i>"; var o = Request.QueryString["AspxErrorPath"]; if (o != null) errPath = o; // Update the UI ErrorPath.InnerHtml = errPath; } }

Although the catalog views are the recommended interface for accessing the SQL Server 2008 catalog, other tools are available as well.

lection of HtmlTableCell elements. The properties that these classes expose let you finely control the appearance of the table and its cells:

download pdf file from server in asp.net c#, c# pdf 417 reader, c# pdf library, itextsharp pdf to excel c#, asp.net upc-a, abcpdf example c#

c# convert pdf to tiff

convert pdf to tiff using ghostscript c# : Create pdf ... - RasterEdge.com
convert pdf to tiff using ghostscript c# : Create pdf signature stamp software Library cloud windows .net wpf class ProgrammingComputerVision_CCdraft27- ...

convert pdf to tiff c# code

How to convert image to pdf using Image Magic in C# | SMART ERP ...
17 Oct 2016 ... This blog will discuss how to convert any type of image file (.jpg, .gif, .tif ..) to pdf . I found a free tool “ ImageMagic .NET”. You can download the ...

B. Incorrect: You cannot tie scheduled tasks to users launching a process. As an alternative, you might create a script that launches both the user s e-mail and the task you need to run and replace the user s e-mail shortcut with the script. C. Incorrect: You cannot tie scheduled tasks to launch when the screen saver starts. However, you could configure a scheduled task to launch at the same idle interval as that used by the screen saver, which would have the same effect. D. Correct: You can configure scheduled tasks to run when the computer is idle. The Windows process that indexes files for easy searching uses this technique. 2. Correct Answer: C A. Incorrect: Task Scheduler is the graphical console for managing scheduled tasks. It cannot be used from a command file. B. Incorrect: At.exe was a command-line tool for scheduling tasks in earlier versions of Windows. C. Correct: SchTasks.exe is the correct tool for managing scheduled tasks from the command prompt or a command file. D. Incorrect: TaskMgr.exe is the Windows Task Manager. It cannot be used from a command file, nor can it be used to manage scheduled tasks. 3. Correct Answers: A, C, and D A. Correct: You can use a scheduled task to start a program. B. Incorrect: You cannot use a scheduled task to directly restart the computer. However, you could create a batch file that called the Shutdown.exe tool and schedule that batch file to run from a scheduled task. C. Correct: You can use Task Scheduler to create a task that sends e-mail messages. D. Correct: You can use Task Scheduler to display a message to the user.

convert pdf to tiff using c#.net

How to convert PDF to TIFF through C - C# Corner
i want convert PDf To Tiff Format in Asp.net or C# . ... to convert pdf to tiff, and this tool also support pdf to multipage tiff . 0 ...

c# convert pdf to tiff free library

Windows 8 Convert PDF file to multipage Tiff in C# - Step by Step ...
21 Mar 2016 ... Convert DOCX file to PDF file in C# (without using MS Office) - Step by Step. ... C# , Silverlight, ASP.NET, Windows Forms, Microsoft Azure, .NET Framework, .NET Framework 4.0.

Your .NET Fram ework solut ions requir e .NET dat a providers t o connect t o dat a sources. These pr ov iders are differ ent fr om t hose used wit h ADO, but t her e are dist inct sim ilar it ies in som e of t he ways y ou use t hem . Wit h .NET dat a prov iders, your solut ions can connect , r ead, and ex ecut e com m ands against dat a sources. The .NET prov iders also offer select ed ot her funct ions, such as t he m anagem ent of input and out put par am et ers, securit y, t ransact ions, and dat abase ser ver errors. Visual St udio .NET ships wit h t wo .NET dat a providers t he SQL Serv er .NET dat a prov ider and t he OLE DB .NET dat a pr ov ider. I n addit ion, y ou can dow nload an ODBC .NET dat a prov ider fr om t he Micr osoft MSDN dow nload sit e ( ht t p: / / m sdn.m icr osoft .com / downloads/ default .asp) .

Slot 2, Offset 0x110, Length 85, DumpStyle BYTE Record Type = PRIMARY_RECORD Record Size = 85 Memory Dump @0x6292C110 00000000: 00000010: 00000020: 00000030: 00000040: 00000050: 30001800 34313520 3534382d 37373233 0...415 548-7723 43413934 373035ff 09000000 05003300 CA94705 .....3. 39003f00 4d005500 3233382d 39352d37 9. .M.U.238-95-7 37363643 6172736f 6e436865 72796c35 766CarsonCheryl5 38392044 61727769 6e204c6e 2e426572 89 Darwin Ln.Ber 6b656c65 79 keley Record Attributes = NULL_BITMAP VARIABLE_COLUMNS

If Today.DayOfWeek = DayOfWeek.Saturday Or Today.DayOfWeek = DayOfWeek.Sunday Then If Not wp.IsInRole( BUILTIN\Backup Operators ) Then On weekends, grant access only to backup operators. Throw New SecurityException( Access denied ) End If End If

c# convert pdf to tiff

How to convert pdf as tiff file in .net - Dotnetspider.com
i have pdf file and i want to show tht pdf as tiff file.is there any code to convert ... pdfsharp.com/PDFsharp/ ... Using 3rd party you can do it very eaisly- ... simple function with which you can convert any PDF file to tiff image in C#.

c# convert pdf to tiff ghostscript

Dot Net: Convert to Tiff to pdf using itextsharp c#
20 May 2015 ... Convert to Tiff to pdf using itextsharp c# // creation of the document with a certain size and certain margins. iTextSharp .text. // creation of the different writers. // load the tiff image and count the total pages. int total = bm.GetFrameCount(System.Drawing.Imaging. document.Open(); iTextSharp .text. pdf . for (int k = ...

.net core barcode, asp.net core barcode generator, asp.net core barcode scanner, c# .net core barcode generator

   Copyright 2020.